:020000040000FA
:06000000703002303A28C6
:08000800A000030EA100831209
:1000100005191028831601178312B23081002B288E
:1000200083160113831203140B190310A80DA90DD5
:10003000AA0DAB0DAC0DAC16FF302C02031D2B2806
:10004000FA302B02031D2B2831152A08AF0029088E
:10005000AE002808AD008B100B11210E8300A00EFE
:04006000200E090065
:0C007400203084008001840A80300402E7
:10008000031C3C281230B000602183160C3085051B
:1000900087018312850187010730990000309A009B
:1000A000103083168E008312603083168F00831207
:1000B0000030831691009F008312C83083168100A0
:1000C000831231309000003083168C008312103080
:1000D0008B00831600309B001C141A088312BC008E
:1000E000831610309B001C141A088312BD009D213A
:1000F00081018E018F010B118B100B108C018B175E
:100100009020311993204221B30B8E2803108519BA
:100110000314B90DF03039020319EB20A021802817
:1001200064003210080031110130B7008B13203009
:10013000370783169B001C141A088312A400103082
:10014000370783169B001C141A088312A300A6000D
:100150000230A6060030370783169B001C141A08CD
:100160008312A200A7000130A7068B17321CBE28FD
:1001700022090339A200A309A409A50924082F0212
:10018000031DE52823082E02031DD32822082D0273
:10019000031DE52801303702031DD3283D18D3285D
:1001A0003D143E14762126082E02031DE52827085B
:1001B0002D02031DE52801303702031DE4283D1CF4
:1001C000E4283D103E149A21E528B70A0230370290
:1001D0000318080096280130B600B300B400B5003B
:1001E000B70085018701B1139020B30B11290310CB
:1001F00085190314B90DF030390203193829B41FD9
:100200008501B41F8701B40B11293708B6080319FB
:10021000B60003190F29FF3085008700B60396301A
:10022000B400311DF4283111321C1B292D0903396A
:10023000AD00AE09AF092F1CF4288E018F010C1CF4
:10024000F4280C102E1EF4288B1320303707BB0027
:100250002F08BA004B2110303707BB002E08BA0018
:100260004B2100303707BB002D08BA004B218B17FC
:1002700085018701B70AB60102303702031CF42852
:100280009D2108003E1C08003E101030BB003D08B8
:10029000BA004B2108008B133A0883161C159A00EC
:1002A00083123B0883169B0055309D00AA309D00A9
:1002B0009C1464009C1859291C1183128B17080088
:1002C000831620309B001C141A088312DF00FF30B5
:1002D000D5000230D6000C30D700BA30D800373005
:1002E000D900DA30DA006F30DB0008000130BD00E1
:1002F0000430C200C5000530C400C600CA00073083
:10030000C100C300C700C800C9005F19C1175F1949
:10031000C2175F19C317DF19C4175F1AC5175F1A11
:10032000C6175F1AC7175F1AC8175F1BC917DF18F0
:10033000CA1708008501870108003D1876210800CA
:1003400001303D05031908005F19A8295C1805163E
:100350005F19AC29DC1885165F19B0295C190514E2
:10036000DF19B429DC1985145F1AB8295C1A8714BF
:100370005F1ABC29DC1A07155F1AC0295C1B071419
:100380005F1AC429DC1B87165F1BC8295D18071676
:10039000DF18CC29DD188715E6300E02031CE4298E
:1003A0005F1D05165F1D85165F1D0514DF1D851475
:1003B0005F1E87145F1E07155F1E07145F1E8716DA
:1003C0005F1F0716DF1C87158F08031908008F01B0
:1003D000850187015508DE00E223D5005608DE00BE
:1003E000E223D6005708DE00551CE223D700580848
:1003F000DE00D51CE223D8005908DE00551DE2239B
:10040000D9005A08DE00D51DE223DA005B08DE00C1
:10041000551EE223DB005F1D272AC11B222AC11CB7
:100420000512C11C162A051258190516CB0B382ABD
:100430005608CB00C101D51BC114D81BC1105818D8
:10044000C110382A0512CB0B382AC103382AC1083B
:10045000031905160319382ACB0B382AD51BC103FB
:100460005508CB00D5185C14D51E5C10D51D5C104A
:100470005F1D542AC21B4F2AC21C8512C21C432A6C
:10048000851258188516CC0B652A5608CC00C20177
:10049000D61BC2145A18C210D619C210652A85126A
:1004A000CC0B652AC203652AC208031985160319F5
:1004B000652ACC0B652AD61BC2035608CC00D61A77
:1004C000DC14561DDC10561FDC105F1D812AC31B77
:1004D0007C2AC31C0510C31C702A05105A19051468
:1004E000CD0B922A5708CD00C301D71BC314D51AD0
:1004F000C310D719C310922A0510CD0B922AC3033B
:10050000922AC308031905140319922ACD0B922AC3
:10051000D71BC3035708CD00571A5C15571F5C1132
:10052000D71D5C11DF1DAE2AC41BA92AC41C85106F
:10053000C41C9D2A8510D51B8514CE0BCA2A5808C9
:10054000CE00C401D81BC414D71AC410D819C410C3
:10055000CA2A8510CE0BCA2AC403CA2ADF1FB92AA9
:10056000CE0BCA2A5808CE00D51BDC15DA1FDC11C9
:10057000CA2AC408031985140319CA2ACE0BCA2A29
:10058000D81BC4035808CE00581ADC15D81FDC113C
:10059000D81DDC115F1EE62AC51BE12AC51C871089
:1005A000C51CD52A8710D51A8714CF0BF72A5908EE
:1005B000CF00C501D91BC514561AC510D81BC510CC
:1005C000F72A8710CF0BF72AC503F72AC5080319A6
:1005D00087140319F72ACF0BF72AD91BC50359082B
:1005E000CF00D91B5C16D91F5C12D91C5C125F1E90
:1005F000132BC61B0E2BC61C0711C61C022B071182
:10060000D71A0715D00B242B5A08D000C601DA1BC5
:10061000C614D51AC610D619C610242B0711D00B34
:10062000242BC603242BC608031907150319242BF2
:10063000D00B242BDA1BC6035A08D0005A1ADC163A
:100640005A1EDC12DA1FDC125F1E402BC71B3B2B2D
:10065000C71C0710C71C2F2B071059190714D10BE3
:10066000512B5B08D100C701DB1BC714D719C7107A
:10067000DB19C710512B0710D10B512BC703512B7E
:10068000C708031907140319512BD10B512BDB1B7E
:10069000C7035B08D100DB195C17DB1D5C135B1E15
:1006A0005C135F1E6D2BC81B682BC81C8712C81CEF
:1006B0005C2B871258198716D20B7E2B5608D20056
:1006C000C801D91BC8145A19C810551AC8107E2B56
:1006D0008712D20B7E2BC8037E2BC80803198716FE
:1006E00003197E2BD20B7E2BD71BC8035908D200CF
:1006F000561ADC17561EDC13DA1FDC135F1F9A2B09
:10070000C91B952BC91C0712C91C892B0712551927
:100710000716D30BB42B5808D300C901D61BC91434
:10072000D91AC910D819C910B42B0712D30BB42B7E
:10073000C903B42B5F1CA52BD30BB42B5708D300D4
:10074000D61B5D14D81F5D10B42BC90803190716FA
:100750000319B42BD30BB42BD51AC9035808D300F3
:10076000D61B5D14D81F5D10DF1CD02BCA1BCB2BF2
:10077000CA1C8711CA1CBF2B8711D51B8715D40B28
:1007800008005508D400CA01D51BCA14561ACA104D
:10079000D619CA1008008711D40B0800CA03080034
:1007A000CA080319871503190800D40B0800D81BC1
:1007B000CA035608D400591ADD14591EDD10DA1F79
:1007C000DD100800C001DE080319DE035E184014C6
:1007D000DE1A40144008C0015E1C4014DE1E4014A6
:0807E000C005C00C5E0C08000E
:084000000D000300040008009C
:02400E00CC33B1
:10420000010078007A007C007E007B0079007F004E
:104210007D007A0078007E007C00FF00FF00FF0038
:104220000100F200F600FA00FE00F200F600FA00CB
:10423000FE00F200F600FA00FE00FF00FF00FF00A3
:10424000030005000500050005000900090009003C
:1042500009000D000D000D000D00FF00FF00FF0024
:10426000FF00FF00FF00FF00FF00FF00FF00FF0056
:10427000FF00FF00FF00FF00FF00FF00FF00FF0046
:10428000FF00FF00FF00FF00FF00FF00FF00FF0036
:10429000FF00FF00FF00FF00FF00FF00FF00FF0026
:1042A000FF00FF00FF00FF00FF00FF00FF00FF0016
:1042B000FF00FF00FF00FF00FF00FF00FF00FF0006
:1042C000FF00FF00FF00FF00FF00FF00FF00FF00F6
:1042D000FF00FF00FF00FF00FF00FF00FF00FF00E6
:1042E000FF00FF00FF00FF00FF00FF00FF00FF00D6
:1042F000FF00FF00FF00FF00FF00FF00FF00DD00E8
:00000001FF
